:020000040000FA
:1000000008030020F9000000FD000000D5000000FA
:1000100000000000000000000000000000000000E0
:1000200000000000000000000000000001010000CE
:1000300000000000000000000301000005010000B6
:100040000701000007010000110600002D06000056
:100050000701000007010000070100000701000080
:10006000FD0A0000190B0000070100000701000055
:10007000350B000007010000070100000701000028
:100080000701000007010000290700000701000028
:100090000701000007010000070100000701000040
:1000A0000701000007010000070100000701000030
:1000B0000701000007010000070100000701000020
:1000C0000348854600F07AF80048004745130000D1
:1000D0000803002004207146084202D0EFF3098093
:1000E00001E0EFF308807146004A10470107000065
:1000F000401EFDD27047000003480047FEE7FEE7C0
:10010000FEE7FEE7FEE7FEE7C100000030B50B4664
:10011000014600202022012409E00D46D5409D42E1
:1001200005D31D469540491B254695404019154667
:10013000521E002DF1DC30BD03460B439B0703D05C
:1001400009E008C9121F08C0042AFAD203E00B789C
:100150000370401C491C521EF9D27047F0B51FB401
:100160000646002082B005464024019100901BE025
:10017000019922460F46304600F042F8049A059B4A
:10018000801A994110D310461946224600F028F8EB
:10019000361A8F410197224601200021009F00F06E
:1001A0001FF838184D4100902046641E0028DFDCFF
:1001B000019B00982946324607B0F0BD064C012548
:1001C000064E05E0E36807CC2B430C3C98471034FF
:1001D000B442F7D3FFF778FFE81A0000081B0000CD
:1001E00010B5202A04DB0146203A9140002010BDC2
:1001F000914020239C1A0346E3401943904010BDD0
:1002000010B5202A04DB0846203AD040002110BD5A
:100210000B46D340D0402024A21A914008431946EF
:1002200010BD00000248016AC2011143016270471B
:1002300000020050C10F8A00044951184A68C306E1
:10024000DB0E0120984002434A60704700020050D4
:10025000F3B58BB00C46FFF7E5FF0B980028744808
:10026000016813D0042211430160102000F0BCF992
:100270000120C00409906F480090042008906E4847
:100280006E49201888420ED800251DE08908890093
:10029000491C0160012000F0A7F90020099068487E
:1002A00000900220EAE767486649201849428842E0
:1002B00002D80125640007E06348634920184942D9
:1002C00088427DD20325A4000026F643089F22E041
:1002D00039460098FFF71AFF5C49844641185C488C
:1002E000814217D2554B02225B1C53486146514351
:1002F000401C0818984209D8A14201D9081B00E007
:10030000601AB04202D2060004920CD05148521C2E
:100310008242EAD97F1C212FDAD900200696C043F9
:100320000190089E54E00999A803084301217A022C
:100330008902511A08430499891E08433C490862FE
:10034000042000F051F9691C79430098FFF7DEFEA4
:10035000049948430DB0F0BD31460098FFF7D6FE32
:100360003A4942183A498A4231D20221324B024676
:100370004A435B1CD7185B429F4224D8A24201D952
:10038000121B00E0A21A019B9A421CD20192069B0A
:100390000F469A4217D10999A80308430121720216
:1003A0008902511A0843B91E0843214908620420F2
:1003B00000F01AF9691C71430098FFF7A7FE00E0EE
:1003C00008E07843C6E7234A491C9142CED9761CFF
:1003D000212EC1D90B9800280FD01F491448016263
:1003E000042000F001F91DA0006803901048016A84
:1003F0000013014203D00020ACE71949EEE70803DF
:1004000001D50C4800E00E488A03A3D40A04920FD9
:1004100003AB9B5CCA058904D20DC90E891C8008F8
:10042000921C59435043FFF771FE800092E7000091
:100430000002005000805101FF1E0AFAFFE0F5059E
:10044000001BB700800F05FDC08782FEFF95E7FF08
:10045000BF77CC000102000018440800010202042A
:1004600016400000044982070A6801D092089200F1
:1004700002430A60704700000002005010B500F00F
:1004800099FA0148006810BD08000020044800687F
:100490008007800F012801D0002070470148704775
:1004A00000020050001BB700044800688007800F5E
:1004B000022801D000207047014870470002005018
:1004C000001BB70008B511A0006800901048016A31
:1004D0000013014201D0002008BD080301D50D48DA
:1004E00000E00D488A03F7D40A04920F6B469B5C28
:1004F000CA058904D20DC90E891C8008921C594373
:100500005043FFF703FE800008BD00000102020413
:100510000002005000805101001BB70008B511A077
:10052000006800901048016A0013014201D00020C9
:1005300008BD080301D50D4800E00D488A03F7D433
:100540000A04920F6B469B5CCA058904D20DC90E42
:10055000891C8008921C59435043FFF7D7FD800047
:1005600008BD000001020204000200500080510199
:10057000001BB70010B5074A93691B091B010B4309
:1005800093611169C908C9000143116100F012FAB1
:1005900010BD00000002005070B5430E1B070DD0C7
:1005A00043009B0F0F4C9B001C192368C5002D0FA7
:1005B000C601F60EB540AB430B432360840A210607
:1005C000090E0DD00103074B890F89000833CB18A2
:1005D00019688005E4B2C00E8440A143114319603C
:1005E00070BD00001002005010B50749074A05E031
:1005F0000B46491E002B01DC002010BDD4680346C9
:10060000A343F5D1012010BD80F520000002005069
:1006100004490420086204484068002800D00047CC
:1006200070470000C04000505800002004490420DA
:10063000086204480068002800D0004770470000A6
:100640004041005058000020024801684908490014
:100650000160704700C000500A492222CA60486009
:10066000012008610869C007FCD10868400606D56A
:1006700008684022104308600020C04370470020F3
:100680007047000000C00050024801680122114379
:100690000160704700C0005005490022CA604860F0
:1006A000012008610869C007FCD188687047000014
:1006B00000C00050054A2123D360506091600120A2
:1006C00010611069C007FCD17047000000C00050E5
:1006D000F0B500230125944603272A469A400A4292
:1006E00009D006685C003A46A2409643224664461A
:1006F0009440264306605B1C082BEED3F0BD00003F
:10070000044603A000F08EFA204601F039F8FEE717
:10071000496E2048617264204661756C742048619E
:100720006E646C65720A000070B50A48C56841695C
:10073000C943C9070AD0084CA068002805D023691E
:10074000E2686169A4682846A04770BD00F006F819
:1007500070BD0000000002406000002041690122DD
:10076000114341617047000070B50C4D0446286884
:100770000A2289005043FFF7C9FC0A21401DFFF7F8
:10078000C5FC401E20612168402211432160810088
:10079000091D2868FFF7BAFC70BD000008000020A2
:1007A0008307FF22DB0E9A408907090E9940002833
:1007B0000BDA0007000F0838830808489B00181858
:1007C000C36993430B43C3617047830804489B008C
:1007D0001B181868904308431860704700ED00E04C
:1007E00000E400E08168082291438160704710B501
:1007F000029C202B00D10023DB000B43134303603A
:1008000001229204914201D110218160214600F021
:1008100001F810BD70B5064619480D4641698906B4
:10082000890F21D040698006800F022823D0FFF76E
:1008300025FE0446A54200D90546002D1ED02946B6
:100840002046FFF763FC401C4008401EFF2800D9EB
:10085000FF207168090A09020143716041002046C6
:10086000891CFFF753FC70BDFFF710FE0400E1D1B7
:10087000FFF71AFEDDE7FFF751FEDAE7002070BD53
:1008800000020050F8B55921304C16228820216012
:10089000226020602368002BF9D02D4D04202860B1
:1008A000FFF7E0FD0820FFF7DDFD1020FFF79CFEBD
:1008B0002869072108432861A86900090001A86187
:1008C0002449A802FFF7C4FC01210220FFF752FED1
:1008D0002148FFF7AFFC214E3046FFF7ABFCB322B7
:1008E000120408213046FFF757FE1D48FFF7A2FC0F
:1008F0001C48FFF79FFC00F05DF81BA0006800900B
:10090000286A291301400025002901D02A4616E053
:10091000010301D5154A00E0154A81030FD40104F3
:10092000890F6B465E5CC3058004C10EDB0D891C1C
:1009300090089B1C71435843FFF7E8FB82000D4E63
:10094000B260FFF79BFDF0602560F8BD000100502C
:100950000002005000E1F505103D80A71CFE23A613
:100960001400C0A71500E0A7010202040080510195
:10097000001BB7001400002010B5592104481622AE
:1009800088230160026003600468002CF9D010BD68
:100990000001005006498A691202FCD408600A2846
:1009A00004D188690002FCD40D2008607047000063
:1009B00000000540F8B520A00068204E0090316A84
:1009C00030131F4C1F4F014201D0002016E00803D6
:1009D00001D5204600E038468A030FD40A04920F5E
:1009E0006B469B5CCA058904D20DC90E891C800820
:1009F000921C59435043FFF789FB8000124D286039
:100A000031694907490F12D0022902D0032910D0B9
:100A10002046B1690907090F491CFFF777FB0B490D
:100A200068604A108018FFF771FBA860F8BD38466F
:100A3000EFE70748EDE70000010202040002005062
:100A400000805101001BB7000400002040420F004D
:100A5000102700000F4A10499042486901D1000A4E
:100A600000E0000B4007400F06D001280ED00228FE
:100A70000ED00A480068704708688007800F012878
:100A800002D00120C00370470548704705487047F1
:100A90000548EFE700000140000200500000002080
:100AA000001BB7001027000008000020F8B513460F
:100AB0000F460646FFF7CEFF044600254008984241
:100AC00001D2022010E0012149068C4202D3032505
:100AD000A40805E0012109068C4201D30125044642
:100AE00019462046FFF712FB2F43376070606D1CDC
:100AF000684301462046FFF709FBF8BD0449012081
:100B0000886004480068002800D000477047000053
:100B1000000001407800002004490120886004485A
:100B20004068002800D000477047000020000140C6
:100B30007800002070B51849CD690022EB05174CEC
:100B40001748002B0BDB0DE00378202B04D20E6836
:100B5000E6545B1C037002E002700B682370CB69E3
:100B6000DB07F1D1AB0515D543888488A34211D2A8
:100B7000002C0FD0094D2035ED5C5B1C45709BB2FD
:100B800043800D60A34205D38280428048680222E0
:100B90009043486070BD000000000540C800002080
:100BA0008000002070B51B4E0D4604467169002080
:100BB00089010322890F2063E260A06000291FD011
:100BC00001291FD0022901D313480068B169090522
:100BD000090F491CFFF79AFA0646002D19D068083C
:100BE00080192946FFF792FA0C49801E88420CD9D9
:100BF000E80080192946FFF789FA0009801E07E0FE
:100C00000748E3E7FFF75EFCE0E703210907084335
:100C1000606270BD0002005000000020FFFF000075
:100C2000001BB7000FB410B503A9044B044A029887
:100C300000F018F810BC08BC04B0184709110000F7
:100C40001000002002E008C8121F08C1002AFAD1D3
:100C500070477047002001E001C1121F002AFBD13C
:100C600070470000FFB58FB00F460446002606E02F
:100C700025280AD0129A11999047641C761C207876
:100C80000028F5D1304613B0F0BD00250121A14A5E
:100C9000009500E00543641C23780846203B9840FB
:100CA0001042F7D120782E2815D104200543607812
:100CB000641C2A280AD101CF641C00900BE0009923
:100CC0000A22514330394018641C009020780146B4
:100CD00030390929F3D920786C280ED004DC4C284F
:100CE00013D06A2812D104E074280ED07A280DD1CE
:100CF0000BE001204005054307E00121090562786A
:100D00000D43824201D16D18641C641C2078864614
:100D100069284AD008DC0028B4D058286DD0632850
:100D200010D0642808D140E070286BD0732812D00E
:100D3000752860D0782860D0129A70461199904733
:100D4000761CE5E03878694608720020487202A8EF
:100D50000190012003E0386801900020C0433F1D4E
:100D600069070CD5002500E06D1C00998D420FDA53
:100D70008542F9DB0199495D0029F5D108E000259C
:100D800000E06D1C8542FCDB0199495D0029F8D12A
:100D9000761907E0019801990078491C0191129A8F
:100DA000119990476D1EF5D2B2E00A200290002101
:100DB0006802400F039102280CD001CFC11784466E
:100DC00000290DDA624608465242002181419446CC
:100DD0002D2008E0FF1DFF08FF0003CF8446EFE74A
:100DE000280504D52B206A46107401203CE0E80752
:100DF0003AD02020F7E70A2000E0102000210391DC
:100E0000029007E0102002900021042005430820F2
:100E1000039100906802400F022810D001CF0021FA
:100E2000844600200D9028071FD5704670280CD0EE
:100E3000029A1020039B42401A430CD015E0FF1D7C
:100E4000FF08FF0003CF8446EBE740206A4610749A
:100E500001200D900CE06046084306D030206A4621
:100E600010747046507402200D907046582804D0BB
:100E700029A001900DA80E900DE02CA0F9E7604686
:100E8000039B029AFFF76AF9019B84469B5C0E9ACA
:100E9000521E0E92137060460843F0D10E9805A9B9
:100EA000081A20300190680701D5009801E0012060
:100EB00000900199884203DD01460198081A00E07C
:100EC00000200025009006E004A8129A405D1199C8
:100ED00090476D1C761C0D988542F5DB04E0129A54
:100EE000302011999047761C0099481E00900029E7
:100EF000F5DC08E00E980E990078491C0E91129AC4
:100F000011999047761C0199481E01900029F1DC47
:100F1000641CB4E6092801003031323334353637E9
:100F20003839616263646566000000003031323335
:100F300034353637383941424344454600000000D5
:100F40000A48016A01221143016205200007416B32
:100F5000074A11404163416B082211434163054830
:100F600041681204114341607047000000000E40C8
:100F7000F7F7FFF7404000500B4908224A620A4A3F
:100F8000403293681B091B019B1D93600A6A012371
:100F9000DB021A430A620A6B1207FCD4096889054E
:100FA000890D01807047000000000E40F8B50D4625
:100FB0000646FFF7E1FCFFF767FB0B4C20680427B0
:100FC0003843206005E03046FFF746FB6D1EADB2AA
:100FD0008036002DF7D12068B8432060FFF734FB3E
:100FE000024900200860F8BD00C000500001005018
:100FF000F7B582B015460E46FFF7BEFCFFF744FB7F
:101000001C4801680422114301600024AF0809E074
:101010000298FFF741FBA10070500298001D641C6C
:10102000A4B20290A742F3D8A004040CAC4214D29C
:101030000298FFF731FB0090684600783055641C39
:10104000A0B2A84209D2694649783154401C80B206
:10105000A84202D2694689783154064801680422C0
:1010600091430160FFF7F0FA03490020086005B0E2
:10107000F0BD000000C0005000010050F7B5002096
:1010800082B0C04315460E460090FFF775FCFFF78F
:10109000FBFA1B4801680422114301600024AF08D9
:1010A00009E0A00031580298FFF704FB0298001DE8
:1010B000641CA4B20290A742F3D8A004000CA8427A
:1010C00012D2315C401C6A4680B21170A84207D22D
:1010D000315C401C80B25170A84201D2305C9070EB
:1010E00000990298FFF7E6FA0548026804218A434E
:1010F0000260FFF7A9FA03490020086005B0F0BDBF
:1011000000C000500001005000B50346FFF742FC4C
:10111000184600BDF0B49C462B4D13466A78294C06
:101120003C265200082816D0182816D020281AD09D
:1011300028281CD010281ED02A46127940281CD0FE
:101140002F46FF78502822D058282CD060460028FF
:1011500007D0F0BC0047A26011E0A878A0600EE0C4
:101160002060F0BC70472068B0431830F8E7206872
:10117000B0432830F4E7521CEDE7012A03D1206880
:10118000B0430830ECE72068B0430C30E8E7921E2B
:10119000A0689742C855E87802D0401CE870F2E792
:1011A000401CE870EBE7A068C855E878401CE87080
:1011B0002068B0431830206001202870002BD0D068
:1011C000F0BC18470000024060000020F0B4184C4A
:1011D0003C26184D082809D018280AD0202810D0FD
:1011E000282812D0002B0AD0F0BC1847687840009D
:1011F00000E0A878A0602068B04308302060F0BC10
:1012000070472068B0431830F8E7E8782B799842A7
:1012100004D0095CA160401CE870ECE72068B04392
:101220001830206001202870002AE8D0F0BC104758
:10123000000002406000002010B51648FEF7FAFFDB
:1012400005200007C16B144A1140C163C16B012224
:1012500012031143C163C16B104A1140C163C16BDA
:10126000012252031143C163C268FF2101310A43C5
:10127000C260C2688A43C2600A4C09492046FFF72F
:1012800073FA2068802108432060C802064908607C
:1012900010BD000008000080EFEFFFFFDFDFFFFF61
:1012A000801A06000000024000E100E0F0B50F4D9A
:1012B000059E2C6840273C432C602C6880273C43CB
:1012C0002C600B4C23716070A1700020E0702070C6
:1012D0000848A060E66006982061626128680821DD
:1012E0008843202108432860F0BD00000000024030
:1012F0006000002015110000F0B50F4D059E2C6810
:1013000040273C432C602C6880273C432C600B4CCE
:1013100023716070A1700020E07020700848A06008
:10132000E6600698206162612868082188432021D0
:1013300008432860F0BD000000000240600000206B
:10134000CD1100001FB5FFF79DFAFFF775FF00F004
:10135000B1F9012000F0B0F8FFF7F2FD00F096F9C6
:1013600000F08CFAFF204949F53000F05DFA48A002
:10137000FFF758FC01214C052046FFF717FE0D2210
:1013800047492046FFF77AFE0D2245492046FFF7E0
:101390002FFE00F075FB3127424D00244048032109
:1013A000183800F08BFA0D213D4800F047FB3C480F
:1013B0000C38FFF7E1FD3A4E1C3E3078401CC0B2BD
:1013C0003070012804D0022807D0032814D10CE083
:1013D0003348C8210838418002E031480838448049
:1013E0002F48083800F020F907E02D48192149015D
:1013F0000838418000F018F934702BA103C900941B
:1014000002AA019403C201230C217620083AFFF7B7
:1014100073FF3E462846FEF76BFE761EFAD2009416
:101420001223234A102176200194FFF73FFF002664
:101430002846FEF75DFE761EFAD2009412231C4A5F
:10144000102176200194FFF731FF00262846FEF791
:101450004FFE761EFAD200941223154A10217620F0
:101460000194FFF723FF00262846FEF741FE761E73
:10147000FAD210480090019030230D4A10217620B6
:10148000FFF714FF72B662B688E700005D17000030
:101490006164632076616C756520697300000000EB
:1014A00030000020086100008902030405000000EC
:1014B0008800002051170000F8B504465920524D0D
:1014C0001622882128602A6029602B68002BF9D019
:1014D0004E48FEF7AFFE4E48FEF7ACFEFFF76AFA45
:1014E00000232B6005221207906B4A490840906345
:1014F000916B012080020143916347498D68092661
:1015000035438D60956B454E35409563956B460030
:10151000354395638D68902635438D60956B404EBD
:1015200035409563956B8600354395638D68092634
:10153000360235438D60956B3A4E35409563956B19
:10154000C600354395638A6809252D032A438A60BE
:101550000D68FF2212029543260235430D604D6847
:1015600007273F02BD4328184860886840004008AC
:101570008860CB627D20C00048610D682D0A2D0275
:1015800025430D604D687027BD4340354D608D6823
:101590006D006D088D608B6208610D682D0A2D024B
:1015A00025430D604C68E408E400241D4C608C6801
:1015B000640064088C604B62C8600C6894433443D8
:1015C0000C604A683C02A2430124A40312194A6039
:1015D0008A68520052088A600B6388618868012219
:1015E00010438860886810221043886088688A15D4
:1015F0001043886088681201104388604B628B62D8
:10160000CB620B63F8BD0000000100501400C0A7BE
:101610001500E0A7FBFBFFFF00000440F7F7FFFF0A
:10162000EFEFFFFFDFDFFFFF30B5174B002204882D
:1016300011469C620488002C1ED0022144881C6341
:1016400045880824002D19D021438488DC628588D0
:101650000424002D14D02143C4885C62C388012077
:10166000002B0FD0014308484030C3699343C36146
:10167000C2690A43C26130BD0222DFE72243E4E7C8
:101680002243E9E70243EEE7000004401CB508A04E
:101690000068019000F00EF82C2000900D23142219
:1016A000032101A800F030F900F0BEF91CBD0000D4
:1016B00023232300F8B505242407206B2063206B27
:1016C00007256D0328432063134841684160134E8A
:1016D0003046FEF7AFFD012210213046FEF75CFFD9
:1016E000012202210E48FEF7F3FF002204210D48DB
:1016F000FEF7EEFF206B284320630B480B4C009055
:101700000823042200212046FFF771F82046FFF746
:1017100069F800202062F8BD400000500C0040A68F
:10172000004000504041005080841E0000000340F3
:101730000649086208680122104308600868C0432F
:10174000C007FBD00869C0B270470000000003402A
:101750000149012048807047140000201CB506494B
:10176000022048800020009001901223034A10219B
:101770007620FFF79BFD1CBD140000208800002090
:1017800010B50446016810A0FFF74CFA11A061687B
:10179000FFF748FA12A0A168FFF744FA13A0E16826
:1017A000FFF740FA14A02169FFF73CFA15A0616920
:1017B000FFF738FA16A0A169FFF734FA17A0E1691C
:1017C000FFF730FA10BD0000723020203D20307845
:1017D00025780A00723120203D20307825780A00D3
:1017E000723220203D20307825780A007233202084
:1017F0003D20307825780A00723132203D20307843
:1018000025780A006C7220203D20307825780A0067
:10181000706320203D20307825780A007073722094
:101820003D20307825780A0070B504460D460F48F3
:10183000FEF700FD22460E4C0121C9062046FFF7A7
:1018400035F9002D0AD0206861030843206048154F
:101850000849086002210820FEF7A2FF064805603B
:101860002068012189070843206070BD020080AE16
:101870000000014000E100E07800002010B50A48B7
:10188000FEF7D8FC0A49094848600A4CE1214902A0
:101890002046FFF787F96068112108436060012046
:1018A00005490003086010BD103D80A70303000038
:1018B000400000500000054000E100E010B5074A7C
:1018C0000023918053800A4601460548FEF734FC08
:1018D0000448416802221143416010BD800000208D
:1018E000E80000200000054010B50021E12000F0D4
:1018F000EBF80021E22000F0E7F810BD10B57021F0
:10190000272000F0E1F810BDFFB50D463EA003C84A
:1019100087B0019100903EA000683EA1049003C9E9
:10192000039102903DA0006805903DA000680690DC
:101930001E465A21532000F0C7F8A521532000F07D
:10194000C3F80124374F02E03846FEF7D1FB641E8E
:10195000FAD2FFF7C9FFFFF7D1FF212E01D20021F4
:1019600000E018213D2000F0AFF80021FD2000F03C
:10197000ABF80321222000F0A7F8A81EC1B2232053
:1019800000F0A2F82520099900F09EF83146312098
:1019900000F09AF83146322000F096F82A463020BE
:1019A000079900F07BF82A462A20079900F076F87C
:1019B000052269463F2000F071F8062202A93A206C
:1019C00000F06CF8012205A9392000F067F8032225
:1019D00004A93E2000F062F8032206A93B2000F093
:1019E0005DF800213C2000F06FF82620109900F0EF
:1019F0006BF80021242000F067F80021212000F07E
:101A000063F80BB0F0BD000012ED679C46000000CB
:101A1000F63F5D004521EF2C5A4000000100000018
:101A20000BDF02000861000010B58F21202000F0BC
:101A30004BF80021FD2000F047F810BD70B50C46B2
:101A400005460021FD2000F03FF84B200001FEF785
:101A50004FFB22462946A02000F020F80748816A63
:101A60000029FCD1FFF74AFF0021E12000F02CF80B
:101A70000021FD2000F028F870BD000080420050D9
:101A800010B58E21202000F01FF80021FD2000F06D
:101A90001BF8F020FEF72CFB10BD0000F8B50F4638
:101AA000084E002115467160FFF742FE002404E055
:101AB000385DFFF73DFE641CE4B2AC42F8D3012070
:101AC0007060F8BD0042005070B50D46054C002115
:101AD0006160FFF72DFE2846FFF72AFE01206060B7
:101AE00070BD000000420050081B000000000020F4
:101AF00088000000440C0000901B000088000020BB
:101B000080020000540C000000805101008051014F
:101B100000000000000000000000000000000000C5
:101B2000123244000000000000000000000000002D
:101B300064009001580220031212121212121212A3
:101B40001312121213121212121212121213121272
:101B50001213121212121212121213121212131262
:101B60000000000000000000000000000000000075
:101B70000000000000000000000000000000000065
:101B80000000000000000000000000000000000055
:04000005000000F9FE
:00000001FF
